 cspddk

 Timestamp is 4da293c2 (Mon Apr 11 17:38:10 2011)

 Preferred load address is 10000000

 Start         Length     Name                   Class
 0001:00000000 00000004H .CRT$XCA                CODE
 0001:00000004 00000004H .CRT$XCZ                CODE
 0001:00000008 00000004H .CRT$XIA                CODE
 0001:0000000c 00000004H .CRT$XIZ                CODE
 0001:00000010 00000004H .CRT$XPA                CODE
 0001:00000014 00000004H .CRT$XPZ                CODE
 0001:00000018 00000004H .CRT$XTA                CODE
 0001:0000001c 00000004H .CRT$XTZ                CODE
 0001:00000020 000002d0H .rdata                  CODE
 0001:000002f0 00000023H .rdata$debug            CODE
 0001:00000314 00002ba4H .text                   CODE
 0001:00002eb8 00000000H .xdata                  CODE
 0001:00002eb8 00000014H .idata$2                CODE
 0001:00002ecc 00000014H .idata$3                CODE
 0001:00002ee0 0000008cH .idata$4                CODE
 0001:00002f6c 0000000cH .idata$6                CODE
 0001:00002f80 000004ebH .edata                  CODE
 0002:00000000 0000008cH .idata$5                DATA
 0002:00000090 00000044H .data                   DATA
 0002:000000e0 00000088H .bss                    DATA
 0003:00000000 000002b8H .pdata                  DATA

  Address         Publics by Value              Rva+Base       Lib:Object

 0000:00000000       ___safe_se_handler_count   00000000     <absolute>
 0000:00000000       ___safe_se_handler_table   00000000     <absolute>
 0001:00000000       __xc_a                     10001000     corelib0:crt0init.obj
 0001:00000004       __xc_z                     10001004     corelib0:crt0init.obj
 0001:00000008       __xi_a                     10001008     corelib0:crt0init.obj
 0001:0000000c       __xi_z                     1000100c     corelib0:crt0init.obj
 0001:00000010       __xp_a                     10001010     corelib0:crt0init.obj
 0001:00000014       __xp_z                     10001014     corelib0:crt0init.obj
 0001:00000018       __xt_a                     10001018     corelib0:crt0init.obj
 0001:0000001c       __xt_z                     1000101c     corelib0:crt0init.obj
 0001:0000003c       ??_C@_1BE@KFLCBOIG@?$AAM?$AAU?$AAT?$AAE?$AAX?$AA_?$AAA?$AAC?$AAR?$AA?$AA@ 1000103c     ddk_mx25_topaz_v1:ddk_sdmav2.obj
 0001:00000050       ??_C@_1BG@GPGAHAMG@?$AAM?$AAU?$AAT?$AAE?$AAX?$AA_?$AAS?$AAD?$AAM?$AAA?$AA?$AA@ 10001050     ddk_mx25_topaz_v1:ddk_sdmav2.obj
 0001:00000278       g_pSdmaBaseRegPA           10001278     ddk_mx25_topaz_v1:soc_ddk_sdma.obj
 0001:0000027c       ??_C@_1BO@ICEODACO@?$AAE?$AAV?$AAE?$AAN?$AAT?$AA_?$AAS?$AAE?$AAT?$AAP?$AAO?$AAI?$AAN?$AAT?$AA?$AA@ 1000127c     ddk_clk:ddk_clk.obj
 0001:0000029c       ??_C@_1CE@KCPPCGKP@?$AAE?$AAV?$AAE?$AAN?$AAT?$AA_?$AAD?$AAV?$AAF?$AAC?$AA_?$AAW?$AAO?$AAR?$AAK?$AAE?$AAR?$AA?$AA@ 1000129c     ddk_clk:ddk_clk.obj
 0001:000002c0       dmaDriverPath              100012c0     ddk_dma:ddk_dma.obj
 0001:000002d8       dmaDriverName              100012d8     ddk_dma:ddk_dma.obj
 0001:00000314       ClockDealloc               10001314 f   ddk_mx25_topaz_v1:soc_ddk_clk.obj
 0001:00000350       DDKClockSetGatingMode      10001350 f   ddk_mx25_topaz_v1:soc_ddk_clk.obj
 0001:000003dc       DDKClockGetGatingMode      100013dc f   ddk_mx25_topaz_v1:soc_ddk_clk.obj
 0001:00000418       DDKClockGetFreq            10001418 f   ddk_mx25_topaz_v1:soc_ddk_clk.obj
 0001:0000041c       DDKClockConfigBaud         1000141c f   ddk_mx25_topaz_v1:soc_ddk_clk.obj
 0001:00000540       DDKClockSetCKO             10001540 f   ddk_mx25_topaz_v1:soc_ddk_clk.obj
 0001:00000588       DDKClockSetpointRequest    10001588 f   ddk_mx25_topaz_v1:soc_ddk_clk.obj
 0001:0000058c       DDKClockSetpointRelease    1000158c f   ddk_mx25_topaz_v1:soc_ddk_clk.obj
 0001:00000590       DDKClockGetSharedConfig    10001590 f   ddk_mx25_topaz_v1:soc_ddk_clk.obj
 0001:000005a0       DDKClockLock               100015a0 f   ddk_mx25_topaz_v1:soc_ddk_clk.obj
 0001:000005ac       DDKClockUnlock             100015ac f   ddk_mx25_topaz_v1:soc_ddk_clk.obj
 0001:000005b8       ClockAlloc                 100015b8 f   ddk_mx25_topaz_v1:soc_ddk_clk.obj
 0001:0000061c       DDKGpioSetConfig           1000161c f   ddk_mx25_topaz_v1:ddk_gpio.obj
 0001:000007b0       DDKGpioGetConfig           100017b0 f   ddk_mx25_topaz_v1:ddk_gpio.obj
 0001:00000888       DDKGpioWriteData           10001888 f   ddk_mx25_topaz_v1:ddk_gpio.obj
 0001:000008ec       DDKGpioWriteDataPin        100018ec f   ddk_mx25_topaz_v1:ddk_gpio.obj
 0001:0000092c       DDKGpioReadData            1000192c f   ddk_mx25_topaz_v1:ddk_gpio.obj
 0001:00000970       DDKGpioReadDataPin         10001970 f   ddk_mx25_topaz_v1:ddk_gpio.obj
 0001:000009c4       DDKGpioReadIntr            100019c4 f   ddk_mx25_topaz_v1:ddk_gpio.obj
 0001:00000a08       DDKGpioReadIntrPin         10001a08 f   ddk_mx25_topaz_v1:ddk_gpio.obj
 0001:00000a5c       DDKGpioClearIntr           10001a5c f   ddk_mx25_topaz_v1:ddk_gpio.obj
 0001:00000a94       DDKGpioClearIntrPin        10001a94 f   ddk_mx25_topaz_v1:ddk_gpio.obj
 0001:00000adc       GpioDealloc                10001adc f   ddk_mx25_topaz_v1:ddk_gpio.obj
 0001:00000b3c       GpioAlloc                  10001b3c f   ddk_mx25_topaz_v1:ddk_gpio.obj
 0001:00000bc8       DDKIomuxSetPinMux          10001bc8 f   ddk_mx25_topaz_v1:soc_ddk_iomux.obj
 0001:00000bf0       DDKIomuxGetPinMux          10001bf0 f   ddk_mx25_topaz_v1:soc_ddk_iomux.obj
 0001:00000c24       DDKIomuxSetPadConfig       10001c24 f   ddk_mx25_topaz_v1:soc_ddk_iomux.obj
 0001:00000c68       DDKIomuxGetPadConfig       10001c68 f   ddk_mx25_topaz_v1:soc_ddk_iomux.obj
 0001:00000cc8       DDKIomuxSetPadConfigPort   10001cc8 f   ddk_mx25_topaz_v1:soc_ddk_iomux.obj
 0001:00000ce8       DDKIomuxGetPadConfigPort   10001ce8 f   ddk_mx25_topaz_v1:soc_ddk_iomux.obj
 0001:00000d0c       DDKIomuxSelectInput        10001d0c f   ddk_mx25_topaz_v1:soc_ddk_iomux.obj
 0001:00000d2c       IomuxDealloc               10001d2c f   ddk_mx25_topaz_v1:soc_ddk_iomux.obj
 0001:00000d60       IomuxAlloc                 10001d60 f   ddk_mx25_topaz_v1:soc_ddk_iomux.obj
 0001:00000dbc       DDKSdmaStartChan           10001dbc f   ddk_mx25_topaz_v1:ddk_sdmav2.obj
 0001:00000e28       DDKSdmaStopChan            10001e28 f   ddk_mx25_topaz_v1:ddk_sdmav2.obj
 0001:00000e70       SdmaDealloc                10001e70 f   ddk_mx25_topaz_v1:ddk_sdmav2.obj
 0001:00000fc0       DDKSdmaUpdateSharedChan    10001fc0 f   ddk_mx25_topaz_v1:ddk_sdmav2.obj
 0001:00001008       DDKSdmaAllocChain          10002008 f   ddk_mx25_topaz_v1:ddk_sdmav2.obj
 0001:00001094       DDKSdmaFreeChain           10002094 f   ddk_mx25_topaz_v1:ddk_sdmav2.obj
 0001:0000113c       DDKSdmaSetBufDesc          1000213c f   ddk_mx25_topaz_v1:ddk_sdmav2.obj
 0001:000011ec       DDKSdmaGetBufDescStatus    100021ec f   ddk_mx25_topaz_v1:ddk_sdmav2.obj
 0001:0000125c       DDKSdmaGetChainStatus      1000225c f   ddk_mx25_topaz_v1:ddk_sdmav2.obj
 0001:00001304       DDKSdmaClearBufDescStatus  10002304 f   ddk_mx25_topaz_v1:ddk_sdmav2.obj
 0001:00001394       DDKSdmaClearChainStatus    10002394 f   ddk_mx25_topaz_v1:ddk_sdmav2.obj
 0001:00001480       SdmaAlloc                  10002480 f   ddk_mx25_topaz_v1:ddk_sdmav2.obj
 0001:00001568       DDKSdmaCloseChan           10002568 f   ddk_mx25_topaz_v1:ddk_sdmav2.obj
 0001:000016b0       DDKSdmaInitChain           100026b0 f   ddk_mx25_topaz_v1:ddk_sdmav2.obj
 0001:000017d0       SdmaInit                   100027d0 f   ddk_mx25_topaz_v1:ddk_sdmav2.obj
 0001:00001980       SdmaDeinit                 10002980 f   ddk_mx25_topaz_v1:ddk_sdmav2.obj
 0001:000019b4       DDKSdmaOpenChan            100029b4 f   ddk_mx25_topaz_v1:ddk_sdmav2.obj
 0001:00001b60       DllEntry                   10002b60 f   ddk_mx25_topaz_v1:cspddk.obj
 0001:00001bcc       Init                       10002bcc f   ddk_mx25_topaz_v1:cspddk.obj
 0001:00001be8       Deinit                     10002be8 f   ddk_mx25_topaz_v1:cspddk.obj
 0001:00001bec       SdmaLoadRamScripts         10002bec f   ddk_mx25_topaz_v1:soc_ddk_sdma.obj
 0001:00001c0c       SdmaSetChanDesc            10002c0c f   ddk_mx25_topaz_v1:soc_ddk_sdma.obj
 0001:00002098       SdmaUpdateChanDesc         10003098 f   ddk_mx25_topaz_v1:soc_ddk_sdma.obj
 0001:000020a0       SdmaSetChanContext         100030a0 f   ddk_mx25_topaz_v1:soc_ddk_sdma.obj
 0001:00002144       BSPClockDealloc            10003144 f   ddk_clk:ddk_clk.obj
 0001:000021c8       BSPClockAlloc              100031c8 f   ddk_clk:ddk_clk.obj
 0001:000022c8       BSPClockGetFreq            100032c8 f   ddk_clk:ddk_clk.obj
 0001:000022ec       BSPClockUpdateFreq         100032ec f   ddk_clk:ddk_clk.obj
 0001:00002388       BSPClockSetGatingModePrepare 10003388 f   ddk_clk:ddk_clk.obj
 0001:00002390       BSPClockSetGatingModeComplete 10003390 f   ddk_clk:ddk_clk.obj
 0001:00002408       BSPClockSetpointRequest    10003408 f   ddk_clk:ddk_clk.obj
 0001:000024bc       BSPClockSetpointRelease    100034bc f   ddk_clk:ddk_clk.obj
 0001:00002508       HalAllocateCommonBuffer    10003508 f   ddk_dma:ddk_dma.obj
 0001:000025cc       HalFreeCommonBuffer        100035cc f   ddk_dma:ddk_dma.obj
 0001:000025e8       MmMapIoSpace               100035e8 f   ddk_map:ddk_map.obj
 0001:000026b0       MmUnmapIoSpace             100036b0 f   ddk_map:ddk_map.obj
 0001:000026c4       StallOneMicrosecond        100036c4 f   ddk_time:ddk_time.obj
 0001:000026fc       StallExecution             100036fc f   ddk_time:ddk_time.obj
 0001:000027c4       BSPSdmaAllocShared         100037c4 f   ddk_sdma:ddk_sdma.obj
 0001:00002874       BSPSdmaAllocChain          10003874 f   ddk_sdma:ddk_sdma.obj
 0001:00002998       BSPSdmaFreeChain           10003998 f   ddk_sdma:ddk_sdma.obj
 0001:00002a00       BSPSdmaBufIntMem           10003a00 f   ddk_sdma:ddk_sdma.obj
 0001:00002a30       BSPSdmaGetM3BaseAddr       10003a30 f   ddk_sdma:ddk_sdma.obj
 0001:00002a38       DeleteCriticalSection      10003a38 f   coredll:COREDLL.dll
 0001:00002a48       LeaveCriticalSection       10003a48 f   coredll:COREDLL.dll
 0001:00002a58       EnterCriticalSection       10003a58 f   coredll:COREDLL.dll
 0001:00002a68       InitializeCriticalSection  10003a68 f   coredll:COREDLL.dll
 0001:00002a78       InterlockedCompareExchange 10003a78 f   coredll:COREDLL.dll
 0001:00002a88       ReleaseMutex               10003a88 f   coredll:COREDLL.dll
 0001:00002a98       WaitForSingleObject        10003a98 f   coredll:COREDLL.dll
 0001:00002aa8       CloseHandle                10003aa8 f   coredll:COREDLL.dll
 0001:00002ab8       CreateMutexW               10003ab8 f   coredll:COREDLL.dll
 0001:00002ac8       Sleep                      10003ac8 f   coredll:COREDLL.dll
 0001:00002ad8       DisableThreadLibraryCalls  10003ad8 f   coredll:COREDLL.dll
 0001:00002ae8       EventModify                10003ae8 f   coredll:COREDLL.dll
 0001:00002af8       CreateEventW               10003af8 f   coredll:COREDLL.dll
 0001:00002b08       InterlockedIncrement       10003b08 f   coredll:COREDLL.dll
 0001:00002b18       InterlockedDecrement       10003b18 f   coredll:COREDLL.dll
 0001:00002b28       FreePhysMem                10003b28 f   coredll:COREDLL.dll
 0001:00002b38       VirtualProtect             10003b38 f   coredll:COREDLL.dll
 0001:00002b48       AllocPhysMem               10003b48 f   coredll:COREDLL.dll
 0001:00002b58       SetLastError               10003b58 f   coredll:COREDLL.dll
 0001:00002b68       VirtualFree                10003b68 f   coredll:COREDLL.dll
 0001:00002b78       VirtualCopy                10003b78 f   coredll:COREDLL.dll
 0001:00002b88       VirtualAlloc               10003b88 f   coredll:COREDLL.dll
 0001:00002b98       QueryPerformanceCounter    10003b98 f   coredll:COREDLL.dll
 0001:00002ba8       QueryPerformanceFrequency  10003ba8 f   coredll:COREDLL.dll
 0001:00002bb8       CacheRangeFlush            10003bb8 f   coredll:COREDLL.dll
 0001:00002bc8       VirtualSetAttributes       10003bc8 f   coredll:COREDLL.dll
 0001:00002bd8       _DllEntryCRTStartup        10003bd8 f   corelib0:pegdentry.obj
 0001:00002c1c       __security_init_cookie     10003c1c f   corelib0:seccinit.obj
 0001:00002c68       __security_check_cookie    10003c68 f   corelib0:armsecgs.obj
 0001:00002c78       __gsfailure                10003c78     corelib0:armsecgs.obj
 0001:00002d7c       _cexit                     10003d7c f   corelib0:cexit.obj
 0001:00002d8c       _initterm                  10003d8c f   corelib0:crt0dat.obj
 0001:00002db8       _cinit                     10003db8 f   corelib0:crt0dat.obj
 0001:00002e18       __crt_ExitProcess          10003e18 f   corelib0:exitproc_proxy.obj
 0001:00002e24       memset                     10003e24 f   corelib1:COREDLL.dll
 0001:00002e34       memcpy                     10003e34 f   corelib1:COREDLL.dll
 0001:00002e44       __rt_udiv                  10003e44 f   corelib1:COREDLL.dll
 0001:00002e54       __security_gen_cookie2     10003e54 f   corelib1:COREDLL.dll
 0001:00002e64       __report_gsfailure         10003e64 f   corelib1:COREDLL.dll
 0001:00002e74       free                       10003e74 f   corelib1:COREDLL.dll
 0001:00002e84       HalTranslateSystemAddress  10003e84 f   ddk_bus:ddk_bus.obj
 0001:00002ea8       TerminateProcess           10003ea8 f   coredll:COREDLL.dll
 0001:00002eb8       __IMPORT_DESCRIPTOR_COREDLL 10003eb8     coredll:COREDLL.dll
 0001:00002ecc       __NULL_IMPORT_DESCRIPTOR   10003ecc     coredll:COREDLL.dll
 0002:00000000       __imp_DeleteCriticalSection 10005000     coredll:COREDLL.dll
 0002:00000004       __imp_LeaveCriticalSection 10005004     coredll:COREDLL.dll
 0002:00000008       __imp_EnterCriticalSection 10005008     coredll:COREDLL.dll
 0002:0000000c       __imp_InitializeCriticalSection 1000500c     coredll:COREDLL.dll
 0002:00000010       __imp_InterlockedCompareExchange 10005010     coredll:COREDLL.dll
 0002:00000014       __imp_ReleaseMutex         10005014     coredll:COREDLL.dll
 0002:00000018       __imp_WaitForSingleObject  10005018     coredll:COREDLL.dll
 0002:0000001c       __imp_CloseHandle          1000501c     coredll:COREDLL.dll
 0002:00000020       __imp_CreateMutexW         10005020     coredll:COREDLL.dll
 0002:00000024       __imp_Sleep                10005024     coredll:COREDLL.dll
 0002:00000028       __imp_DisableThreadLibraryCalls 10005028     coredll:COREDLL.dll
 0002:0000002c       __imp_EventModify          1000502c     coredll:COREDLL.dll
 0002:00000030       __imp_CreateEventW         10005030     coredll:COREDLL.dll
 0002:00000034       __imp_InterlockedIncrement 10005034     coredll:COREDLL.dll
 0002:00000038       __imp_InterlockedDecrement 10005038     coredll:COREDLL.dll
 0002:0000003c       __imp_FreePhysMem          1000503c     coredll:COREDLL.dll
 0002:00000040       __imp_VirtualProtect       10005040     coredll:COREDLL.dll
 0002:00000044       __imp_AllocPhysMem         10005044     coredll:COREDLL.dll
 0002:00000048       __imp_SetLastError         10005048     coredll:COREDLL.dll
 0002:0000004c       __imp_VirtualFree          1000504c     coredll:COREDLL.dll
 0002:00000050       __imp_VirtualCopy          10005050     coredll:COREDLL.dll
 0002:00000054       __imp_VirtualAlloc         10005054     coredll:COREDLL.dll
 0002:00000058       __imp_QueryPerformanceCounter 10005058     coredll:COREDLL.dll
 0002:0000005c       __imp_QueryPerformanceFrequency 1000505c     coredll:COREDLL.dll
 0002:00000060       __imp_CacheRangeFlush      10005060     coredll:COREDLL.dll
 0002:00000064       __imp_VirtualSetAttributes 10005064     coredll:COREDLL.dll
 0002:00000068       __imp_memset               10005068     corelib1:COREDLL.dll
 0002:0000006c       __imp_memcpy               1000506c     corelib1:COREDLL.dll
 0002:00000070       __imp___rt_udiv            10005070     corelib1:COREDLL.dll
 0002:00000074       __imp___rt_sdiv64by64      10005074     corelib1:COREDLL.dll
 0002:00000078       __imp___security_gen_cookie2 10005078     corelib1:COREDLL.dll
 0002:0000007c       __imp___report_gsfailure   1000507c     corelib1:COREDLL.dll
 0002:00000080       __imp_free                 10005080     corelib1:COREDLL.dll
 0002:00000084       __imp_TerminateProcess     10005084     coredll:COREDLL.dll
 0002:00000088       \177COREDLL_NULL_THUNK_DATA 10005088     coredll:COREDLL.dll
 0002:00000090       g_DmaAdapter               10005090     ddk_mx25_topaz_v1:ddk_sdmav2.obj
 0002:000000a0       g_SupportBothEdgeIntr      100050a0     ddk_mx25_topaz_v1:soc_ddk_gpio.obj
 0002:000000a4       g_MaxPort                  100050a4     ddk_mx25_topaz_v1:soc_ddk_gpio.obj
 0002:000000a8       g_PhyBaseAddress           100050a8     ddk_mx25_topaz_v1:soc_ddk_gpio.obj
 0002:000000c8       g_hDma                     100050c8     ddk_dma:ddk_dma.obj
 0002:000000cc       __security_cookie          100050cc     corelib0:seccinit.obj
 0002:000000d0       __security_cookie_complement 100050d0     corelib0:seccinit.obj
 0002:000000e0       g_pCRM                     100050e0     ddk_mx25_topaz_v1:soc_ddk_clk.obj
 0002:000000e4       g_pDdkClkConfig            100050e4     ddk_mx25_topaz_v1:soc_ddk_clk.obj
 0002:000000f4       g_pHostSharedUA            100050f4     ddk_mx25_topaz_v1:ddk_sdmav2.obj
 0002:000000f8       g_pHostSharedPA            100050f8     ddk_mx25_topaz_v1:ddk_sdmav2.obj
 0002:000000fc       g_HostSharedSize           100050fc     ddk_mx25_topaz_v1:ddk_sdmav2.obj
 0002:00000120       _exitflag                  10005120     corelib0:cexit.obj
 0002:00000130       g_pGPIO                    10005130     <common>
 0002:00000140       g_csDdkClk                 10005140     <common>
 0002:00000154       g_fStallCounterSet         10005154     <common>
 0002:00000158       g_StallCounter             10005158     <common>
 0002:0000015c       g_StallDummy               1000515c     <common>
 0002:00000160       __onexitend                10005160     <common>
 0002:00000164       __onexitbegin              10005164     <common>

 entry point at        0001:00002bd8

 Static symbols

 0001:00000ef4       SdmaSetChanOverride        10001ef4 f   ddk_mx25_topaz_v1:ddk_sdmav2.obj
 0001:00000f84       SdmaValidChan              10001f84 f   ddk_mx25_topaz_v1:ddk_sdmav2.obj
 0001:00002cbc       doexit                     10003cbc f   corelib0:cexit.obj
